Archive member included because of file (symbol)

e:/winavr-20071221/bin/../lib/gcc/avr/4.2.2/avr5\libgcc.a(_divmodhi4.o)
                              ks0108.o (__divmodhi4)
e:/winavr-20071221/bin/../lib/gcc/avr/4.2.2/avr5\libgcc.a(_exit.o)
                              e:/winavr-20071221/bin/../lib/gcc/avr/4.2.2/../../../../avr/lib/avr5/crtm16.o (exit)
e:/winavr-20071221/bin/../lib/gcc/avr/4.2.2/avr5\libgcc.a(_copy_data.o)
                              AD_prevod.o (__do_copy_data)
e:/winavr-20071221/bin/../lib/gcc/avr/4.2.2/avr5\libgcc.a(_clear_bss.o)
                              AD_prevod.o (__do_clear_bss)
e:/winavr-20071221/bin/../lib/gcc/avr/4.2.2/avr5\libgcc.a(_udivmodhi4.o)
                              e:/winavr-20071221/bin/../lib/gcc/avr/4.2.2/avr5\libgcc.a(_divmodhi4.o) (__udivmodhi4)
e:/winavr-20071221/bin/../lib/gcc/avr/4.2.2/../../../../avr/lib/avr5\libc.a(itoa.o)
                              AD_prevod.o (itoa)
e:/winavr-20071221/bin/../lib/gcc/avr/4.2.2/../../../../avr/lib/avr5\libc.a(strrev.o)
                              e:/winavr-20071221/bin/../lib/gcc/avr/4.2.2/../../../../avr/lib/avr5\libc.a(itoa.o) (strrev)

Allocating common symbols
Common symbol       size              file

ks0108FontColor     0x1               ks0108.o
ks0108Coord         0x3               ks0108.o
ks0108FontRead      0x2               ks0108.o
ks0108Font          0x2               ks0108.o

Memory Configuration

Name             Origin             Length             Attributes
text             0x00000000         0x00020000         xr
data             0x00800060         0x0000ffa0         rw !x
eeprom           0x00810000         0x00010000         rw !x
fuse             0x00820000         0x00000400         rw !x
lock             0x00830000         0x00000400         rw !x
signature        0x00840000         0x00000400         rw !x
*default*        0x00000000         0xffffffff

Linker script and memory map

LOAD e:/winavr-20071221/bin/../lib/gcc/avr/4.2.2/../../../../avr/lib/avr5/crtm16.o
LOAD AD_prevod.o
LOAD ks0108.o
LOAD touch.o
LOAD e:/winavr-20071221/bin/../lib/gcc/avr/4.2.2/avr5\libgcc.a
LOAD e:/winavr-20071221/bin/../lib/gcc/avr/4.2.2/../../../../avr/lib/avr5\libc.a
LOAD e:/winavr-20071221/bin/../lib/gcc/avr/4.2.2/avr5\libgcc.a

.hash
 *(.hash)

.dynsym
 *(.dynsym)

.dynstr
 *(.dynstr)

.gnu.version
 *(.gnu.version)

.gnu.version_d
 *(.gnu.version_d)

.gnu.version_r
 *(.gnu.version_r)

.rel.init
 *(.rel.init)

.rela.init
 *(.rela.init)

.rel.text
 *(.rel.text)
 *(.rel.text.*)
 *(.rel.gnu.linkonce.t*)

.rela.text
 *(.rela.text)
 *(.rela.text.*)
 *(.rela.gnu.linkonce.t*)

.rel.fini
 *(.rel.fini)

.rela.fini
 *(.rela.fini)

.rel.rodata
 *(.rel.rodata)
 *(.rel.rodata.*)
 *(.rel.gnu.linkonce.r*)

.rela.rodata
 *(.rela.rodata)
 *(.rela.rodata.*)
 *(.rela.gnu.linkonce.r*)

.rel.data
 *(.rel.data)
 *(.rel.data.*)
 *(.rel.gnu.linkonce.d*)

.rela.data
 *(.rela.data)
 *(.rela.data.*)
 *(.rela.gnu.linkonce.d*)

.rel.ctors
 *(.rel.ctors)

.rela.ctors
 *(.rela.ctors)

.rel.dtors
 *(.rel.dtors)

.rela.dtors
 *(.rela.dtors)

.rel.got
 *(.rel.got)

.rela.got
 *(.rela.got)

.rel.bss
 *(.rel.bss)

.rela.bss
 *(.rela.bss)

.rel.plt
 *(.rel.plt)

.rela.plt
 *(.rela.plt)

.text           0x00000000     0x1cbe
 *(.vectors)
 .vectors       0x00000000       0x54 e:/winavr-20071221/bin/../lib/gcc/avr/4.2.2/../../../../avr/lib/avr5/crtm16.o
                0x00000000                __vectors
                0x00000000                __vector_default
 *(.vectors)
 *(.progmem.gcc*)
 *(.progmem*)
 .progmem.data  0x00000054      0xc24 AD_prevod.o
                0x00000c78                . = ALIGN (0x2)
                0x00000c78                __trampolines_start = .
 *(.trampolines)
 .trampolines   0x00000c78        0x0 linker stubs
 *(.trampolines*)
                0x00000c78                __trampolines_end = .
 *(.jumptables)
 *(.jumptables*)
 *(.lowtext)
 *(.lowtext*)
                0x00000c78                __ctors_start = .
 *(.ctors)
                0x00000c78                __ctors_end = .
                0x00000c78                __dtors_start = .
 *(.dtors)
                0x00000c78                __dtors_end = .
 SORT(*)(.ctors)
 SORT(*)(.dtors)
 *(.init0)
 .init0         0x00000c78        0x0 e:/winavr-20071221/bin/../lib/gcc/avr/4.2.2/../../../../avr/lib/avr5/crtm16.o
                0x00000c78                __init
 *(.init0)
 *(.init1)
 *(.init1)
 *(.init2)
 .init2         0x00000c78        0xc e:/winavr-20071221/bin/../lib/gcc/avr/4.2.2/../../../../avr/lib/avr5/crtm16.o
 *(.init2)
 *(.init3)
 *(.init3)
 *(.init4)
 .init4         0x00000c84       0x16 e:/winavr-20071221/bin/../lib/gcc/avr/4.2.2/avr5\libgcc.a(_copy_data.o)
                0x00000c84                __do_copy_data
 .init4         0x00000c9a       0x10 e:/winavr-20071221/bin/../lib/gcc/avr/4.2.2/avr5\libgcc.a(_clear_bss.o)
                0x00000c9a                __do_clear_bss
 *(.init4)
 *(.init5)
 *(.init5)
 *(.init6)
 *(.init6)
 *(.init7)
 *(.init7)
 *(.init8)
 *(.init8)
 *(.init9)
 .init9         0x00000caa        0x8 e:/winavr-20071221/bin/../lib/gcc/avr/4.2.2/../../../../avr/lib/avr5/crtm16.o
 *(.init9)
 *(.text)
 .text          0x00000cb2        0x4 e:/winavr-20071221/bin/../lib/gcc/avr/4.2.2/../../../../avr/lib/avr5/crtm16.o
                0x00000cb2                __vector_1
                0x00000cb2                __vector_12
                0x00000cb2                __bad_interrupt
                0x00000cb2                __vector_6
                0x00000cb2                __vector_3
                0x00000cb2                __vector_11
                0x00000cb2                __vector_13
                0x00000cb2                __vector_17
                0x00000cb2                __vector_19
                0x00000cb2                __vector_7
                0x00000cb2                __vector_4
                0x00000cb2                __vector_9
                0x00000cb2                __vector_2
                0x00000cb2                __vector_15
                0x00000cb2                __vector_8
                0x00000cb2                __vector_14
                0x00000cb2                __vector_10
                0x00000cb2                __vector_16
                0x00000cb2                __vector_18
                0x00000cb2                __vector_20
 .text          0x00000cb6      0x100 AD_prevod.o
                0x00000cb6                __vector_5
                0x00000cd8                main
 .text          0x00000db6      0xd32 ks0108.o
                0x00000f06                ks0108GotoXY
                0x00001354                ks0108Puts
                0x00001516                ks0108SetInverted
                0x00000f50                ks0108DoReadData
                0x00000db6                ks0108ReadFontData
                0x00001856                ks0108DrawRect
                0x00000fec                ks0108WriteData
                0x00000e6c                ks0108StringWidth_P
                0x00001536                ks0108FillRect
                0x000010d4                ks0108PutChar
                0x000013f4                ks0108InvertRect
                0x0000165e                ks0108Init
                0x000016ae                ks0108DrawRoundRect
                0x00000dd4                ks0108CharWidth
                0x00000ee0                ks0108WriteCommand
                0x00000fdc                ks0108ReadData
                0x00000e40                ks0108StringWidth
                0x00000dbe                ks0108SelectFont
                0x000013a2                ks0108SetDot
                0x00000ea0                ks0108Enable
                0x00001304                ks0108Puts_P
                0x000018a6                ks0108DrawLine
 .text          0x00001ae8      0x124 touch.o
                0x00001ae8                read_adc
                0x00001af6                F_radek
                0x00001b1e                F_stlaceno
 .text          0x00001c0c        0x0 e:/winavr-20071221/bin/../lib/gcc/avr/4.2.2/avr5\libgcc.a(_divmodhi4.o)
 .text          0x00001c0c        0x0 e:/winavr-20071221/bin/../lib/gcc/avr/4.2.2/avr5\libgcc.a(_exit.o)
 .text          0x00001c0c        0x0 e:/winavr-20071221/bin/../lib/gcc/avr/4.2.2/avr5\libgcc.a(_copy_data.o)
 .text          0x00001c0c        0x0 e:/winavr-20071221/bin/../lib/gcc/avr/4.2.2/avr5\libgcc.a(_clear_bss.o)
 .text          0x00001c0c        0x0 e:/winavr-20071221/bin/../lib/gcc/avr/4.2.2/avr5\libgcc.a(_udivmodhi4.o)
 .text          0x00001c0c       0x42 e:/winavr-20071221/bin/../lib/gcc/avr/4.2.2/../../../../avr/lib/avr5\libc.a(itoa.o)
                0x00001c0c                itoa
 .text          0x00001c4e       0x20 e:/winavr-20071221/bin/../lib/gcc/avr/4.2.2/../../../../avr/lib/avr5\libc.a(strrev.o)
                0x00001c4e                strrev
                0x00001c6e                . = ALIGN (0x2)
 *(.text.*)
 .text.libgcc   0x00001c6e       0x26 e:/winavr-20071221/bin/../lib/gcc/avr/4.2.2/avr5\libgcc.a(_divmodhi4.o)
                0x00001c6e                __divmodhi4
                0x00001c6e                _div
 .text.libgcc   0x00001c94        0x0 e:/winavr-20071221/bin/../lib/gcc/avr/4.2.2/avr5\libgcc.a(_exit.o)
 .text.libgcc   0x00001c94        0x0 e:/winavr-20071221/bin/../lib/gcc/avr/4.2.2/avr5\libgcc.a(_copy_data.o)
 .text.libgcc   0x00001c94        0x0 e:/winavr-20071221/bin/../lib/gcc/avr/4.2.2/avr5\libgcc.a(_clear_bss.o)
 .text.libgcc   0x00001c94       0x28 e:/winavr-20071221/bin/../lib/gcc/avr/4.2.2/avr5\libgcc.a(_udivmodhi4.o)
                0x00001c94                __udivmodhi4
                0x00001cbc                . = ALIGN (0x2)
 *(.fini9)
 .fini9         0x00001cbc        0x0 e:/winavr-20071221/bin/../lib/gcc/avr/4.2.2/avr5\libgcc.a(_exit.o)
                0x00001cbc                exit
                0x00001cbc                _exit
 *(.fini9)
 *(.fini8)
 *(.fini8)
 *(.fini7)
 *(.fini7)
 *(.fini6)
 *(.fini6)
 *(.fini5)
 *(.fini5)
 *(.fini4)
 *(.fini4)
 *(.fini3)
 *(.fini3)
 *(.fini2)
 *(.fini2)
 *(.fini1)
 *(.fini1)
 *(.fini0)
 .fini0         0x00001cbc        0x2 e:/winavr-20071221/bin/../lib/gcc/avr/4.2.2/avr5\libgcc.a(_exit.o)
 *(.fini0)
                0x00001cbe                _etext = .

.data           0x00800060        0x0 load address 0x00001cbe
                0x00800060                PROVIDE (__data_start, .)
 *(.data)
 .data          0x00800060        0x0 e:/winavr-20071221/bin/../lib/gcc/avr/4.2.2/../../../../avr/lib/avr5/crtm16.o
 .data          0x00800060        0x0 AD_prevod.o
 .data          0x00800060        0x0 ks0108.o
 .data          0x00800060        0x0 touch.o
 .data          0x00800060        0x0 e:/winavr-20071221/bin/../lib/gcc/avr/4.2.2/avr5\libgcc.a(_divmodhi4.o)
 .data          0x00800060        0x0 e:/winavr-20071221/bin/../lib/gcc/avr/4.2.2/avr5\libgcc.a(_exit.o)
 .data          0x00800060        0x0 e:/winavr-20071221/bin/../lib/gcc/avr/4.2.2/avr5\libgcc.a(_copy_data.o)
 .data          0x00800060        0x0 e:/winavr-20071221/bin/../lib/gcc/avr/4.2.2/avr5\libgcc.a(_clear_bss.o)
 .data          0x00800060        0x0 e:/winavr-20071221/bin/../lib/gcc/avr/4.2.2/avr5\libgcc.a(_udivmodhi4.o)
 .data          0x00800060        0x0 e:/winavr-20071221/bin/../lib/gcc/avr/4.2.2/../../../../avr/lib/avr5\libc.a(itoa.o)
 .data          0x00800060        0x0 e:/winavr-20071221/bin/../lib/gcc/avr/4.2.2/../../../../avr/lib/avr5\libc.a(strrev.o)
 *(.data*)
 *(.rodata)
 *(.rodata*)
 *(.gnu.linkonce.d*)
                0x00800060                . = ALIGN (0x2)
                0x00800060                _edata = .
                0x00800060                PROVIDE (__data_end, .)

.bss            0x00800060        0xa load address 0x00001cbe
                0x00800060                PROVIDE (__bss_start, .)
 *(.bss)
 .bss           0x00800060        0x0 e:/winavr-20071221/bin/../lib/gcc/avr/4.2.2/../../../../avr/lib/avr5/crtm16.o
 .bss           0x00800060        0x1 AD_prevod.o
                0x00800060                j
 .bss           0x00800061        0x1 ks0108.o
                0x00800061                ks0108Inverted
 .bss           0x00800062        0x0 touch.o
 .bss           0x00800062        0x0 e:/winavr-20071221/bin/../lib/gcc/avr/4.2.2/avr5\libgcc.a(_divmodhi4.o)
 .bss           0x00800062        0x0 e:/winavr-20071221/bin/../lib/gcc/avr/4.2.2/avr5\libgcc.a(_exit.o)
 .bss           0x00800062        0x0 e:/winavr-20071221/bin/../lib/gcc/avr/4.2.2/avr5\libgcc.a(_copy_data.o)
 .bss           0x00800062        0x0 e:/winavr-20071221/bin/../lib/gcc/avr/4.2.2/avr5\libgcc.a(_clear_bss.o)
 .bss           0x00800062        0x0 e:/winavr-20071221/bin/../lib/gcc/avr/4.2.2/avr5\libgcc.a(_udivmodhi4.o)
 .bss           0x00800062        0x0 e:/winavr-20071221/bin/../lib/gcc/avr/4.2.2/../../../../avr/lib/avr5\libc.a(itoa.o)
 .bss           0x00800062        0x0 e:/winavr-20071221/bin/../lib/gcc/avr/4.2.2/../../../../avr/lib/avr5\libc.a(strrev.o)
 *(.bss*)
 *(COMMON)
 COMMON         0x00800062        0x8 ks0108.o
                0x00800062                ks0108FontColor
                0x00800063                ks0108Coord
                0x00800066                ks0108FontRead
                0x00800068                ks0108Font
                0x0080006a                PROVIDE (__bss_end, .)
                0x00001cbe                __data_load_start = LOADADDR (.data)
                0x00001cbe                __data_load_end = (__data_load_start + SIZEOF (.data))

.noinit         0x0080006a        0x0
                0x0080006a                PROVIDE (__noinit_start, .)
 *(.noinit*)
                0x0080006a                PROVIDE (__noinit_end, .)
                0x0080006a                _end = .
                0x0080006a                PROVIDE (__heap_start, .)

.eeprom         0x00810000        0x0
 *(.eeprom*)
                0x00810000                __eeprom_end = .

.fuse
 *(.fuse)
 *(.lfuse)
 *(.hfuse)
 *(.efuse)

.lock
 *(.lock*)

.signature
 *(.signature*)

.stab           0x00000000      0x378
 *(.stab)
 .stab          0x00000000      0x378 e:/winavr-20071221/bin/../lib/gcc/avr/4.2.2/../../../../avr/lib/avr5/crtm16.o

.stabstr        0x00000000       0x5f
 *(.stabstr)
 .stabstr       0x00000000       0x5f e:/winavr-20071221/bin/../lib/gcc/avr/4.2.2/../../../../avr/lib/avr5/crtm16.o

.stab.excl
 *(.stab.excl)

.stab.exclstr
 *(.stab.exclstr)

.stab.index
 *(.stab.index)

.stab.indexstr
 *(.stab.indexstr)

.comment
 *(.comment)

.debug
 *(.debug)

.line
 *(.line)

.debug_srcinfo
 *(.debug_srcinfo)

.debug_sfnames
 *(.debug_sfnames)

.debug_aranges  0x00000000       0x60
 *(.debug_aranges)
 .debug_aranges
                0x00000000       0x20 AD_prevod.o
 .debug_aranges
                0x00000020       0x20 ks0108.o
 .debug_aranges
                0x00000040       0x20 touch.o

.debug_pubnames
                0x00000000      0x286
 *(.debug_pubnames)
 .debug_pubnames
                0x00000000       0x30 AD_prevod.o
 .debug_pubnames
                0x00000030      0x21c ks0108.o
 .debug_pubnames
                0x0000024c       0x3a touch.o

.debug_info     0x00000000      0xc41
 *(.debug_info)
 .debug_info    0x00000000      0x14b AD_prevod.o
 .debug_info    0x0000014b      0xa0e ks0108.o
 .debug_info    0x00000b59       0xe8 touch.o
 *(.gnu.linkonce.wi.*)

.debug_abbrev   0x00000000      0x383
 *(.debug_abbrev)
 .debug_abbrev  0x00000000       0xeb AD_prevod.o
 .debug_abbrev  0x000000eb      0x210 ks0108.o
 .debug_abbrev  0x000002fb       0x88 touch.o

.debug_line     0x00000000      0xe3c
 *(.debug_line)
 .debug_line    0x00000000      0x1ae AD_prevod.o
 .debug_line    0x000001ae      0xac4 ks0108.o
 .debug_line    0x00000c72      0x1ca touch.o

.debug_frame    0x00000000      0x1e0
 *(.debug_frame)
 .debug_frame   0x00000000       0x30 AD_prevod.o
 .debug_frame   0x00000030      0x170 ks0108.o
 .debug_frame   0x000001a0       0x40 touch.o

.debug_str      0x00000000      0x38d
 *(.debug_str)
 .debug_str     0x00000000       0xce AD_prevod.o
                                0x102 (size before relaxing)
 .debug_str     0x000000ce      0x298 ks0108.o
                                0x366 (size before relaxing)
 .debug_str     0x00000366       0x27 touch.o
                                 0xe0 (size before relaxing)

.debug_loc      0x00000000      0xc84
 *(.debug_loc)
 .debug_loc     0x00000000       0x1e AD_prevod.o
 .debug_loc     0x0000001e      0xc66 ks0108.o

.debug_macinfo
 *(.debug_macinfo)
OUTPUT(AD_prevod.elf elf32-avr)
LOAD linker stubs
